:100000000C94A0010C94BD010C94BD010C94861AB3
:100010000C94BD010C94BD010C94BD010C94BD0168
:100020000C94BD010C94BD010C94A5210C94772275
:100030000C94901C0C94BD010C94BD010C94BD015A
:100040000C94BD010C94BD010C94BD010C94BD0138
:100050000C94BD010C94341D0C94BD010C94BD0195
:100060000C94BD010C94BD010C94BD010C94BD0118
:100070000C94BD010C94BD010C94BD010C94BD0108
:100080000C94BD010C94BD010C94BD010C94BD01F8
:100090000C94BD010C94BD010C94BD010C94BD01E8
:1000A0000C94BD010C94BD010C94BD016D046D0454
:1000B0009904990401051F05370637062A05C3056B
:1000C000D405D405E4220B2303240B230324572354
:1000D0007A230324D123E0232300220021002000DF
:1000E0001F001E0035001C001700150008001A0034
:1000F00014002B002F000A0009000700160004005E
:10010000E0002C000500190006001B001D00E100A6
:100110000000E300E20029000000000000002300CE
:1001200024002500260027002D002E001C001800AA
:100130000C00120013002F00300030000B000D00E7
:100140000E000F00330034002800110010003600AC
:1001500037003800310000000151E6002A0000009D
:10016000000000003F003E003D003C003B003A0024
:100170000100010001000100010001000100010077
:100180000100010001000100010001000100010067
:100190000100010001000100010001000000010058
:1001A000010001000000000000003F00400041008D
:1001B000420043004400450001000100010001002D
:1001C00001000100010001004E004B000100010090
:1001D0000100460001005000510052004F004A004B
:1001E0004D000000010001004C0000000000000074
:1001F0001403730070006100720072006F007700DA
:100200003600320000002C034100740073007500BA
:100210007300680069005F004D006F0072006900A4
:100220006D006F0074006F005F00370034007400D1
:10023000680000000403090409023B00020100A059
:10024000FA09040000010301010009211101000164
:100250002240000705810308000109040100010391
:10026000000000092111010001227B000705820323
:10027000200001120100020000000874DA6174011C
:10028000000102000105010902A10185020901A185
:100290000005091901290815002501950875018136
:1002A000020501093009311581257F950275088104
:1002B0000609381581257F950175088106050C0A08
:1002C00038021581257F950175088106C0C005019A
:1002D0000980A101850319012AB700150126B7007D
:1002E000950175108100C0050C0901A10185041953
:1002F000012AA002150126A002950175108100C0F7
:1003000005010906A101050719E029E715002501E6
:10031000950875018102950175088101050719008D
:1003200029FF150026FF00950675088100050819AC
:10033000012905950575019102950175039101C08B
:1003400011241FBECFEFDAE0DEBFCDBF11E0A0E089
:10035000B1E0E2EAF9E402C005900D92A23AB107D9
:10036000D9F722E0A2EAB1E001C01D92A13BB20799
:10037000E1F70E94F7140C94CF240C94000081E064
:10038000089581E008950C94C10108950C94C5016D
:100390001F93CF93DF9300D000D01F92CDB7DEB76D
:1003A00049835A836B833091A50189819A813111E8
:1003B00014C0662359F0222349F00E947408182FB4
:1003C000682F89819A810E941D0803C00E944808F5
:1003D000182F69817A81812F04C00E947408698175
:1003E0007A810F900F900F900F900F90DF91CF9127
:1003F0001F910C94830FFC01262F40815181628153
:10040000738184810C94C80181E00895CF93DF93B8
:10041000EC0160E00E94FB01BE01DF91CF910C94E2
:10042000C6010C9407110C94031108950E94C7068D
:100430000E9415022FEF84E39CE021508040904001
:10044000E1F700C000000C945A1D0F931F93CF9347
:10045000DF938C0161E00E94FB01EC01B8010E9476
:10046000C3018823F1F1B801CE010E9491198823BC
:10047000C1F1B801CE010E94A517882391F1B801FE
:10048000CE010E94ED18882361F1F8018281882352
:1004900009F1CB358DE5D807C1F050F4C115FCE565
:1004A000DF0781F0CF3DDC45A9F40E94910D19C012
:1004B000CC35EDE5DE0761F0CD35DD4559F40E9420
:1004C000D40C08C00E9416020CC00E94DD0C02C0B1
:1004D0000E94E00CC801DF91CF911F910F910C9405
:1004E000BF0180E0DF91CF911F910F9108950E948D
:1004F000731C0C9490020E9493020C94791C089532
:100500000C947F0281E008950C9482020895CF93A9
:10051000C82F0E9480028C2F0E948402CF910895E0
:1005200080E00C9487020E94B11B0C9487020E9409
:10053000B11B9091A401891721F08093A4010C9420
:1005400087020895CF93DF93CDB7DEB72B970FB611
:10055000F894DEBF0FBECDBF4F83588769877A8777
:100560008B8761110E94200C9E012F5F3F4F86E018
:10057000F90111928A95E9F785E0FE013796D901D4
:1005800001900D928A95E1F789819A814C815D8174
:10059000452B31F09F3F31F491E08F3F19F403C0B8
:1005A00091E001C090E090FF09C049815A816B81C0
:1005B0007C818D819E810E94410B05C0C9010E94F2
:1005C00004028111F2CF2B960FB6F894DEBF0FBE56
:1005D000CDBFDF91CF910895FC01808191810E9470
:1005E000B6080895CF93882309F4A4C0C82F823891
:1005F000C1F40E94B11B81FD9DC069E3809102019D
:10060000909103010E944B1C0E94420C2FEF81EE3F
:1006100094E0215080409040E1F700C0000069E381
:1006200019C0833801F50E94B11B80FD83C063E5CA
:1006300080910201909103010E944B1C0E94420C88
:100640002FEF81EE94E0215080409040E1F700C010
:10065000000063E580910201909103010E944D1C0E
:10066000CF910C94420C8438C1F40E94B11B82FDDE
:1006700061C067E480910201909103010E944B1CCC
:100680000E94420C2FEF81EE94E021508040904078
:10069000E1F700C0000067E4DDCF8CEF8C0F813AFA
:1006A000D0F46C2F80910201909103010E94151CDF
:1006B000882349F06C2F80910201909103010E94E0
:1006C0004D1C0E94420C6C2F8091020190910301FD
:1006D0000E944B1CC5CF80E28C0F883048F4C77055
:1006E00081E001C0880FCA95EAF70E94030CB8CFD9
:1006F000EBE5EC0FE33040F4F0E0E05AFE4F808190
:1007000090E0CF910C94DD1BE8E5EC0FE73150F45D
:10071000F0E0EE0FFF1FEE5CFE4F80819181CF91E4
:100720000C94F31BCD3E30F08C2F0E947C15CF91A2
:100730000C944E16CF910895882309F464C0823832
:1007400079F40E94B11B81FF5EC069E380910201D0
:10075000909103010E944B1C0E94420C69E310C05F
:100760008338B1F40E94B11B80FF4DC063E58091D6
:100770000201909103010E944B1C0E94420C63E510
:1007800080910201909103010E944D1C0C94420C37
:10079000843879F40E94B11B82FF35C067E48091F0
:1007A0000201909103010E944B1C0E94420C67E4DD
:1007B000E7CF9CEF980F913A10F4682FE1CF90E2C9
:1007C000980F983050F4877091E001C0990F8A9586
:1007D000EAF7892F0E94090CD9CF9BE5980F933037
:1007E00020F480E090E00C94DD1B98E5980F9731A1
:1007F00020F480E090E00C94F31B8D3E20F00E94EA
:10080000D7150C944E1608951F93CF93DF93182F8E
:10081000EB010E94F202209741F08FE99FE00197DF
:10082000F1F700C000002197F6CF812FDF91CF9123
:100830001F910C949C03893319F060E070E002C0B2
:1008400060E570E00C940404882321F00E94030CFE
:100850000C94420C0895882321F00E94090C0C94FA
:10086000420C0895CF92DF92EF92FF920F931F9365
:10087000CF93DF937C01D62FC72FFC011281058116
:1008800002950F700E94F90B8823B9F01123A9F08B
:100890008C2F807F803421F080E28D0F883068F0CB
:1008A0008091890282FD09C082E00E94A20C0E9410
:1008B000F90B91E0D82ED92601C0D12CCC2EC294B0
:1008C0008FE0C8228C2D90E08C30910508F0CFC1CC
:1008D000FC01EA5AFF4F0C945D248C2F807FCF706F
:1008E000882311F0C295C07F112399F0CC2309F41D
:1008F000AAC180E28D0F883010F0D11104C08C2F76
:100900000E94030C03C08C2F0E94130C0E94420C07
:100910009AC18D2F0E949C03CC2309F4A8C180E2C8
:100920008D0F883038F1DD2329F18C2F0E94190CAE
:1009300024C08C2F807FCF70803211F0C295C07F91
:10094000DD2319F0D130A1F13DC08091890282FFF1
:1009500017C0112349F0CC2329F08C2F0E94030CDF
:100960000E94420C80E070C180E00E949C03CC2376
:1009700009F47DC18C2F0E94090C0E94420C77C1A2
:10098000112371F0002341F0013031F40E94230C57
:100990008C2B0E942B0C6BC10E94230C8C2B1DC036
:1009A000002319F0013009F462C10E94380C25C0FF
:1009B000112321F0063008F05AC10EC0053008F0AE
:1009C00056C11BC0112361F0002331F0F70185816E
:1009D00080FF39C18F7085838C2F0E94240447C10A
:1009E000002359F0D93309F03FC1FFEF07EE13E0C0
:1009F000F15000401040E1F735C18C2F0E942B04CC
:100A000036C18C2F86958695837019F0813061F000
:100A10002EC1112321F08D2F9C2F937002C080E0F6
:100A200090E00E94DD1B2BC1112321F08D2F9C2F04
:100A3000937002C080E090E00E94F31B20C18D2FD4
:100A4000112319F00E947C1502C00E94D7150E9444
:100A50004E1615C18C2F837009F047C011110BC1C0
:100A60002D2F229526952770220F220F6D2F6F7044
:100A7000862F90E0A0E0B0E0022E04C0880F991FFE
:100A8000AA1FBB1F0A94D2F7D4FF10C04FE050E05A
:100A900060E070E004C0440F551F661F771F2A9561
:100AA000D2F7409550956095709503C040E050E0B6
:100AB000BA01C695C695C3708A019B01082B192BF4
:100AC0002A2B3B2BC901B801C23049F058F4C13080
:100AD00019F00E943307CFC00E942107CCC00E94AA
:100AE0004507C9C00E941F07C6C0112319F08C2FEB
:100AF000817001C08695882309F4BDC02D2F2295F1
:100B000026952770220F220F6D2F6F70862F90E091
:100B1000A0E0B0E0022E04C0880F991FAA1FBB1FDF
:100B20000A94D2F7D4FF10C04FE050E060E070E0CC
:100B300004C0440F551F661F771F2A95D2F74095B2
:100B400050956095709503C040E050E0BA01C6959D
:100B5000C695C3708A019B01082B192B2A2B3B2BAE
:100B6000C901B801C23049F058F4C13019F00E94EF
:100B7000F80781C00E94E6077EC00E940A087BC079
:100B80000E94590778C0CF70112339F08C2F0E9432
:100B90007F078D2F0E9424046EC08D2F0E942B048E
:100BA0008C2F0E94A00767C0D23F21F128F4D03FCC
:100BB00041F0D13FC1F043C0D33F19F1D43F79F0A8
:100BC0003EC0112341F0053008F051C08C2F8F71C9
:100BD0000E94C5074CC0063008F049C0F7CF80918D
:100BE000890282FF18C0112339F08C2F8F710E9467
:100BF0007F073DC01123C9F38C2F8F710E94A0077E
:100C000036C0112329F08C2F8F710E946A072FC0E4
:100C10000E9465072CC0112349F0CF718C2F0E94D0
:100C20007F0763E08C2F0E94870C21C081E00E9427
:100C3000A20C0230E0F082E00E94A20C18C0112346
:100C400031F0002391F28D2F0E94F20210C0002398
:100C500099F2D93349F41FEF27EE33E011502040C9
:100C60003040E1F700C000008D2F0E949C0388EF08
:100C70008C0D843020F40E94B11B0E948702DD207D
:100C8000C9F00E94F50B80FD15C0F70112820E9489
:100C9000EF0B0E947F07C7010E947B060E94EF0BAB
:100CA000DF91CF911F910F91FF90EF90DF90CF9048
:100CB0000C94A007DF91CF911F910F91FF90EF90BF
:100CC000DF90CF9008950F931F93CF93DF93EC01A4
:100CD000688179818A810E94C1088C010E941C0868
:100CE0000E940D07B801CE010E943204DF91CF911E
:100CF0001F910F910895CF93DF93EC019881898123
:100D00002B813C81232B31F08F3F31F481E09F3FD9
:100D100019F403C081E001C080E080FD1DC0CE0158
:100D20000E942502811110C00E94F90B8823A1F0B6
:100D30008A81882389F08091890282FD0DC082E03A
:100D4000DF91CF910C94A20CCE010E946306CE01DC
:100D5000DF91CF910C940602DF91CF91089580E04E
:100D600090E00E94DD1B80E090E00E94F31B0E9457
:100D7000200C0E94420C0E947F170C944E1680910A
:100D80000201909103010E944F1C0C94AF060E9437
:100D9000100C0C94BF0692959F70963079F010F469
:100DA000925001C09A50923068F4803F69F018F474
:100DB000883E40F409C0843F29F406C0883E20F0F4
:100DC000813F11F080E0089581E00895FC01808169
:100DD00091810E94B6080E94CB060895CF93DF93BD
:100DE00000D000D01F92CDB7DEB70F900F900F90BC
:100DF0000F900F90DF91CF910895CF93DF9300D0A4
:100E000000D000D0CDB7DEB726960FB6F894DEBF7F
:100E10000FBECDBFDF91CF910895089508950C9432
:100E20000E070C940F070E9411076093D70170936F
:100E3000D8018093D9019093DA010C94AF060C94F9
:100E400013070F931F930091D7011091D8012091A0
:100E5000D9013091DA01602B712B822B932B1F91DA
:100E60000F910C9413070F931F930091D7011091CA
:100E7000D8012091D9013091DA01602371238223B6
:100E800093231F910F910C9413070F931F930091BD
:100E9000D7011091D8012091D9013091DA01602752
:100EA0007127822793271F910F910C9413070C949D
:100EB0000E070E9457076093D3017093D40180936B
:100EC000D5019093D6010C94AF0660E070E0CB01A1
:100ED0000C9459070F931F9341E050E060E070E0DD
:100EE0008A019B0104C0000F111F221F331F8A9526
:100EF000D2F7C901B8011F910F910C9459070F93B4
:100F00001F9341E050E060E070E004C0440F551FC3
:100F1000661F771F8A95D2F78091D3019091D401F3
:100F2000A091D501B091D6018A019B01082B192B04
:100F30002A2B3B2BC901B8011F910F910C94590723
:100F40000F931F9341E050E060E070E004C0440F55
:100F5000551F661F771F8A95D2F74095509560956B
:100F600070958091D3019091D401A091D501B09159
:100F7000D6018A019B01082319232A233B23C90197
:100F8000B8011F910F910C9459070F931F9341E0E3
:100F900050E060E070E004C0440F551F661F771FEB
:100FA0008A95D2F78091D3019091D401A091D50177
:100FB000B091D6018A019B01082719272A273B27D0
:100FC000C901B8011F910F910C9459070F931F93FA
:100FD0000091D3011091D4012091D5013091D60117
:100FE000602B712B822B932B1F910F910C9459071F
:100FF0000F931F930091D3011091D4012091D5013B
:101000003091D60160237123822393231F910F9186
:101010000C9459070F931F930091D3011091D401A1
:101020002091D5013091D60160277127822793271F
:101030001F910F910C945907089527E0929F800DFE
:101040001124E82FE695E695E695877051E001C0FA
:10105000550F8A95EAF785E0E89FF0011124EA55DB
:10106000FE4F20E030E070E04081CB01022E02C054
:10107000969587950A94E2F7817081958427852358
:10108000842781932F5F3F4F2530310569F70895FD
:1010900027E0929F800D1124682F669566956695CE
:1010A000982F977085E0689FB001112440E050E0D0
:1010B00080E0FB01E40FF51FEA55FE4F208130E090
:1010C000092E02C0369527950A94E2F7217033273E
:1010D000042E01C0220F0A94EAF7822B4F5F5F4F64
:1010E0004530510531F70895BF92CF92DF92EF92CC
:1010F000FF920F931F93CF93DF938C01C090D30186
:10110000D090D401E090D501F090D6018091D70124
:101110009091D801A091D901B091DA01C82AD92AB9
:10112000EA2AFB2ACFE1D0E0D701C6010C2E04C089
:10113000B695A795979587950A94D2F780FD04C038
:10114000219790F7B12C07C0BC2EB8018C2F0E94BC
:10115000960F0197A9F38B2DDF91CF911F910F91DE
:10116000FF90EF90DF90CF90BF900895CF93DF93E3
:10117000EC010E947408BE010E94960FDF91CF918E
:1011800008951F93CF93DF93EB019091A5019923CD
:1011900021F0CB010E94B60813C0882349F0CB018F
:1011A0000E947408182F682FCE010E941D0804C0E9
:1011B000CB010E944808182FBE01812F0E94960F74
:1011C000DF91CF911F9108951F93CF93DF93C0912B
:1011D000DB0116E08091DC01C81799F0D0E01C9F7C
:1011E000F0011D9FF00D1124E352FE4F408151810B
:1011F00062817381848195810E94FD062196C7706A
:10120000E9CFDF91CF911F91089540910D02509148
:101210000E0260910F027091100280911102909164
:1012200012020C94FD06EF92FF920F931F93CF933F
:10123000DF938091120282958F7009F065C08091D2
:101240000F02882309F460C08091DB01F090DC017B
:1012500010910D0200910E02609110027091110226
:1012600091E01F3F09F090E0C0910001D091010191
:10127000292F96E0E92E8F1509F446C061157105F6
:1012800021F00F3F21F030E003C031E001C0322FE8
:1012900090E030FD36C0E89EF001E99EF00D11248B
:1012A000DF01A352BE4F11963C911197301329C014
:1012B0003C91311326C012963C911297311121C0F6
:1012C00013964D915C911497461B570B4C175D0775
:1012D000C0F4809112028F70806180931202EE51EF
:1012E000FE4F80818F70806180838DE092E00E944C
:1012F0007B06DF91CF911F910F91FF90EF900C949F
:10130000E40801968770B7CFDF91CF911F910F91BD
:10131000FF90EF9008959F92AF92BF92CF92DF928D
:10132000EF92FF920F931F93CF93DF93CDB7DEB76A
:1013300061970FB6F894DEBF0FBECDBF8C0185E07C
:10134000F801DE011D9601900D928A95E1F7D80112
:101350001296EC9090910D02E0910E0220911002F5
:10136000309111022115310531F0EF3F31F481E068
:101370009F3F19F403C081E001C080E0B82FB17035
:101380009B2E80FD2DC1D8014C9111965C91119737
:101390001396AD90BC9014978DE0C82E82E0D82EA5
:1013A000F0900F02B501621B730B20910001309188
:1013B0000101FF2009F4E5C0809112026217730752
:1013C00008F0A1C0282F207F09F052C05E1313C07F
:1013D000491311C0FE2CE1100EC08F708061809304
:1013E00012020E940509C6010E947B06809112022A
:1013F000F801858333C1AB2831F05F3F31F481E0E0
:101400004F3F19F403C081E001C080E080FD03C0BC
:1014100081E08E2502C080E090E0F82FF170FF2E71
:1014200080FF1CC08091DB012091DC0136E0821737
:1014300009F4F1C090E0389FF001399FF00D1124BC
:10144000E352FE4F6181561306C06081461303C00C
:101450006281E61203C001968770E9CFFE2CEE2070
:1014600009F4FCC08091120281608093120260C076
:101470005E1312C0491310C0E1100EC0F80185833D
:10148000C8010E947B0686E0F801ADE0B2E0019061
:101490000D928A95E1F7BCC0C8010E94E606882338
:1014A00061F1EE2051F120911202822F82958F700E
:1014B00090E0029774F080910D0290910E0298874F
:1014C0008F831986BB86AA862C87CE0107960E9439
:1014D0007B0686E0F801ADE0B2E001900D928A95BE
:1014E000E1F70E9413090E9405090AC05E1711F175
:1014F000C8010E94E60681112CC0C8010E947B062B
:10150000FF24F394ABC0282F207F81F77A2DB98A6E
:10151000A88A6E2D89890E94EE068DE092E00E94D5
:101520007B0686E0D6011D928A95E9F70E9405099F
:10153000F12C94C04913DCCFE110DACFF801858398
:10154000C8010E947B0686E0D6011D928A95E9F7C4
:1015500085C0EE2091F220911202822F82958F7029
:1015600090E002970CF4B5CF80910D0290910E029D
:101570009A8389831B82BD82AC822E83CE01019621
:10158000A6CF62177307F8F4FE2CEE2009F4B5CF4E
:101590005E130BC0491309C086E0F801ADE0B2E06C
:1015A00001900D928A95E1F759C0C8010E94E606A4
:1015B00081118FCF80911202816080931202C80145
:1015C0000E947B064BC07A2DB98AA88A6E2D898924
:1015D0000E94EE0686E0F60111928A95E9F718C09E
:1015E000EE2009F48ACFC8010E94E606F82E88236F
:1015F00009F483CF86E0F801ADE0B2E001900D92EE
:101600008A95E1F78DE092E00E94EC020E941309B6
:101610000E94050923C04D875E878D859E850E94A7
:10162000B608292F22952F70223028F49F7039F0A8
:10163000811105C00BC0243028F49F7049F4805EEE
:10164000883020F0C8010E947B069F2CF92C06C030
:10165000D80115969C91907F91F7F8CF8F2D6196C8
:101660000FB6F894DEBF0FBECDBFDF91CF911F91B3
:101670000F91FF90EF90DF90CF90BF90AF909F9031
:1016800008951F93CF93DF93CDB7DEB72C970FB696
:10169000F894DEBF0FBECDBF4F83588769877A8726
:1016A0008B879C87CE0107960E948B098823D1F0F7
:1016B0009F8188852A853B85232B31F08F3F31F42C
:1016C00081E09F3F19F403C081E001C080E080FD0C
:1016D00047C04F81588569857A858B859C850E9496
:1016E000FD063EC086E0FE013796DE0111960190B0
:1016F0000D928A95E1F7FF81E8856A857B85611502
:10170000710531F0EF3F31F481E0FF3F19F403C080
:1017100081E001C080E080FD23C02091DC0130E049
:10172000C9010196877099274091DB0150E0841729
:101730009507F1F1F983EA837D836C8396E0929FAC
:10174000D001939FB00D1124A352BE4FFE013196DC
:1017500001900D929A95E1F78093DC010E94E408D4
:1017600016E08091DB019091DC01891771F1189FDF
:10177000C001112483529E4F0E948B09882329F1B6
:10178000E091DB011E9FF0011124E352FE4F4081E6
:10179000518162817381848195810E94FD068091CF
:1017A000DB0190E00196877099278093DB01D9CF08
:1017B0000E94C7061092DC011092DB01EDE0F2E01E
:1017C00086E0DF011D928A95E9F72C960FB6F89412
:1017D000DEBF0FBECDBFDF91CF911F9108958091E5
:1017E0001B02859585958595089580911B028770CC
:1017F000089590911B02977081E009F480E00895AC
:1018000080912602089590912602892B80932602CA
:101810000895809590912602892380932602089549
:1018200010922602089590912502892B809325021B
:10183000089580959091250289238093250208952B
:1018400010922502089580911C02089508950C9429
:10185000260C0C94270C9091890292FD08C090915F
:101860001C02981721F080931C020C94290C0895F7
:1018700080911C02882329F010921C0280E00C94B5
:10188000290C0895CF93DF93E0910201F0910301B9
:10189000809126028083E0910201F0910301908102
:1018A00080912502892B808380911C02882381F0FE
:1018B000E0910201F09103019081892B8083809156
:1018C0000201909103010E94091C81110E94380CB1
:1018D000C0910201D091030148E050E063E172E061
:1018E000CE010E947724892B69F088E0FE01A3E1F4
:1018F000B2E001900D928A95E1F7CE01DF91CF9190
:101900000C94C41BDF91CF9108950C94260C9091F8
:10191000890292FD10C098E0899F90011124262B26
:1019200020931B020E947F0780911B02859585955D
:1019300085950C94850C0C947F0710921B0280E017
:101940000C94850C20911B028095822380931B02AE
:10195000982F977099F430E0482F082E000C550B03
:101960002417350759F09091890292FD07C085959B
:10197000859585950E94A0070C949D0C08959091E3
:10198000890292FB222720F9281769F080FB92F93F
:101990009093890280918802909189020E940D0D96
:1019A00082E00C94A20C08958091890282FB882722
:1019B00080F991E089270C94BF0C81E00C94BF0C56
:1019C00080E00C94BF0C6FEF7FEF80E090E00C9410
:1019D000B92480E090E00E94952421E0893E9E4F4A
:1019E00009F020E0822F089582E090E00C948D248D
:1019F00083E090E00C948D24CF9384E090E00E94EB
:101A00008D24C82F82E290E00E948D242C2F30E09C
:101A1000A901582BCA01CF910895CF93C92F682FE0
:101A200084E090E00E949B246C2F82E290E0CF91B2
:101A30000C949B24AB01BC018FE090E00C94AD248E
:101A4000AB01BC0183E190E00C94AD2460E070E058
:101A5000CB010C94200D60E070E0CB010E941A0DC8
:101A60000C94260D69EE7EEF80E090E00E94B92490
:101A700060E082E090E00E949B2460E083E090E0E0
:101A80000E949B241092D7011092D8011092D90184
:101A90001092DA0160E084E090E00E949B2460E014
:101AA00082E290E00E949B2460E085E090E00E944A
:101AB0009B2460E086E090E00E949B246FEF87E02B
:101AC00090E00E949B2440E050E0BA0188E090E062
:101AD0000E94AD2460E08DE090E00E949B2440E0F5
:101AE00050E0BA0188E190E00E94AD2460E087E117
:101AF00090E00E949B2440E050E0BA018CE190E02D
:101B00000E94AD2460E070E080E290E00E94B92481
:101B100040E050E0BA0188E190E00E94AD240C94CE
:101B20002B0D0C94320D682F8EE090E00C949B24CA
:101B30000E94FD1C60933502709336028093370239
:101B40009093380260933102709332028093330293
:101B500090933402089585B7806885BF85B7806803
:101B600085BF08950C94C11208950C94B40D0C9483
:101B7000B40D0C94B70D0C94B40D0C94BB0D0C94D7
:101B8000B40D0E94AB0D83EB90E10E94A71B0E9455
:101B9000BF0D0C94BD0D0E94B50D0C94B40D0E94A8
:101BA000CD100C9486020E94E81C0E9472100E94C4
:101BB000D9120E940C120E94CF0D0E948D170E9414
:101BC000E3120C94B90D8F929F92AF92BF92CF9275
:101BD000DF92EF92FF920F931F93CF93DF93CDB7D6
:101BE000DEB72A970FB6F894DEBF0FBECDBF0E94B6
:101BF0003012982E81110E94980D87E2A82E82E063
:101C0000B82E00E010E0802E802F0E94F110D82E18
:101C1000F501C1905F01C826B1F40F5F1F4F0A3074
:101C2000110589F78FEF89838A831B820E94F11C3B
:101C30008160782F9D838C8349815A816B818D814E
:101C40000E94A2022FC08091390281FD0E94F710EC
:101C5000E12CFF24F3948C2D8F21F1F00E94B20D22
:101C6000882399F0EE828F82DF2081E009F480E002
:101C700088870E94F11C8160782F9A8789874E811E
:101C80005F8168858A850E94A202F801E95DFD4FA7
:101C90008081F826F08206C0E394FF0CF7E0EF1293
:101CA000DACFBBCF81E0911001C080E02A960FB659
:101CB000F894DEBF0FBECDBFDF91CF911F910F9182
:101CC000FF90EF90DF90CF90BF90AF909F908F905C
:101CD00008950E94E30D0E94C1120E946C160C949C
:101CE0009702CF93DF930E949B0FEC01811521E5B2
:101CF000920708F045C0811530E5930708F094C0BD
:101D0000883E910528F5803E910508F0F8C0883A94
:101D1000910570F4853A910508F07CC081309105F9
:101D200009F475C008F4E8C0049708F0E8C0E4C0FE
:101D30008F3B910508F0E0C0C85AD0E0CC0FDD1F02
:101D4000CD59DE4F0990D881C02DCE019464D8C002
:101D5000811540E2940758F4811551E0950708F089
:101D6000CEC08D3E910508F4C7C09065C9C0C115AD
:101D700080E4D80708F4C0C0DF70CE01906AC0C00C
:101D8000811525E59207A8F4811534E5930708F03D
:101D900095C0811543E5940708F07BC0811552E595
:101DA000950708F061C0D82FCC27CE01816F906ACB
:101DB000A7C0C11589E5D807A0F4C11528E5D20749
:101DC00008F082C0C11536E5D30708F095C08C2F06
:101DD0000E942F108F7190E0D82FCC27CE019062F7
:101DE0008FC0C1154AE5D40708F474C0CE019056DF
:101DF0008115904208F080C08D2F8F710E942F10A6
:101E0000DD27D0628F71AE01582BCA0179C081E005
:101E100090E076C0C55AD0E0CF56DE4F8881C82FFB
:101E2000D0E0CE0190646CC074E0969587957A9569
:101E3000E1F7282F23703C2F337081E090E002C03F
:101E4000880F991F3A95E2F79C68AC01522B9A01D2
:101E50009C2F9F709695969550E2959FE0011124D6
:101E6000C9018C2B9D2B4CC08370992721E030E059
:101E700002C0220F331F8A95E2F79C2F9695969504
:101E800080E2989FE0011124C22BD32BCE019C68E5
:101E900037C08370992721E030E002C0220F331F42
:101EA0008A95E2F79C2F9695969540E2949FE001E3
:101EB0001124C22BD32BCE019A6822C0D82FCC2755
:101EC000CE01846F906A1CC0DC2FCC27CE01806FBE
:101ED000906A16C08C2F8F700E942F1094E0D695B8
:101EE000C7959A95E1F7CF70D0E0DC2FCC27D06969
:101EF0009E01282BC90104C080E090E001C0CE0102
:101F0000DF91CF91089526E4829FC0011124FC0146
:101F100027E0729FE00DF11D1124E60FF11DEE0F79
:101F2000FF1FE852FF4F8591949108950E94830FFF
:101F30000E94710E08958238910569F1B0F48133E1
:101F4000910509F46DC048F48932910509F463C024
:101F50008A32910509F469C008958533910509F421
:101F600055C089339105B9F00895833E910569F113
:101F700038F4803E9105B1F0823E910509F1089553
:101F8000863E9105A9F1873E9105B9F1843E910500
:101F900009F064C023C02091880220FD4FC021FDBC
:101FA0004DC008958091880280FD44C080918902CF
:101FB00080FF44C08091880284FD42C083EE4DC002
:101FC0008091880282FF38C0F5CF8091880282FD1F
:101FD00033C08091890280FD31C0ECCF80918902AD
:101FE00081FF32C08091880284FD2AC087EE35C00F
:101FF0008091880283FF26C0F5CF8091880283FDFF
:1020000021C08091890281FD1FC0ECCF80918802A0
:1020100085FD1CC01DC08091880285FD19C016C0B9
:102020008091880286FD16C017C08091880286FDC7
:1020300013C010C089E311C082EE0FC080EE0DC046
:1020400080E00BC086EE09C084EE07C089E205C0BF
:1020500085E303C08AE201C081E390E00895909196
:10206000880292FF0DC0282F2871283019F4877F2D
:10207000846006C0282F2471243011F48B7F88607F
:1020800093FF0DC0282F2871283119F4877E8461B1
:1020900006C0282F2471243111F48B7E8861209191
:1020A000890220FF0DC0382F3871383019F4877F2E
:1020B000816006C0382F3171313011F48E7F886015
:1020C00021FF0DC0282F2871283119F4877E8161E6
:1020D00006C0282F2171213111F48E7E886194FD74
:1020E000877E0895109284021092850210928602D3
:1020F000109287020895CF92DF92EF92FF926B01C8
:102100007C010E94C11281110EC00E94FD1CC61AE2
:10211000D70AE80AF90AC0928402D0928502E092B6
:102120008602F0928702FF90EF90DF90CF900895A3
:102130000F931F930E94C112882321F01F910F91CA
:102140000C94FD1C0E94FD1C0091840210918502DC
:102150002091860230918702600F711F821F931FAA
:102160001F910F91089580E008950C94E30C0E9454
:1021700030128FE39CE90197F1F700C000000E9444
:10218000301280E00E94F11080FF04C00E94B51060
:102190000C945A1D08950C94B7100E94E90C8111FB
:1021A00002C00E94910D0E94F40C809339020E949B
:1021B000FC0C90938902809388020E94CB100E94AD
:1021C000F80C682F70E080E090E00E941F0760919B
:1021D000D3017091D4018091D5019091D6010C94D6
:1021E0005707E82FF0E0EB56FD4F808108950895E2
:1021F00080EA8A95F1F7089500C008950C94F810CC
:1022000008950C9400110C9401110C9400110C947D
:1022100005110C940011FF920F931F93CF93DF933E
:1022200000D000D01F92CDB7DEB70E94C1126091DE
:102230009F028823E9F185E0F82E8E010F5F1F4F82
:10224000F8018F2D11928A95E9F7862F90E0B80159
:102250008B569D4F0E94F112882389F080918A024B
:1022600090E045E050E0B8018B569D4F0E947724E6
:1022700021E020933A02892B61F410E016C080918E
:102280003A028823D1F3F8011192FA94E9F71092F7
:102290003A02A0918A02B0E0AB56BD4F85E0F8014A
:1022A00001900D928A95E1F711E00E9413020DC092
:1022B00070E06B567D4F80918A0290E08B569D4F67
:1022C0000E947B130E94091110E0812F0F900F9044
:1022D0000F900F900F90DF91CF911F910F91FF9072
:1022E0000895F894E82FE295EF70F0E031A1282FDF
:1022F0002F7081E090E001C0880F2A95EAF7982FAF
:102300009095932391A392A1892B82A37894089509
:102310000F931F93CF93DF93CBE9D1E089918F3F48
:1023200011F00E94711181E0C03AD807B9F7C4E9F1
:10233000D1E00BE911E089918F3F11F00E947111FA
:102340000C171D07C1F7DF91CF911F910F910895D1
:10235000CF92DF92EF92FF920F931F93CF93DF9371
:102360008C01C62FD0E0CE0185569E4F7C01FC012A
:1023700090819F3F09F447C0D62EF894E92FE2954B
:10238000EF70F0E081A19F7021E030E001C0220FEA
:102390009A95EAF7822B81A382A12095282322A374
:1023A00078940E94FC10E4E9F1E04BE951E031E05F
:1023B000C12C21912F3F89F0A22FA295AF70B0E0E0
:1023C00090968C9190E02F7002C0959587952A95F4
:1023D000E2F780FD02C0832F01C080E0C82A330FDE
:1023E0004E175F0731F7F70180818F3F11F00E9490
:1023F000711161E0C11001C060E08D2D0E94FE10DE
:10240000C00FD11FC882DF91CF911F910F91FF9014
:10241000EF90DF90CF9008958091040180910401A6
:10242000811102C095E001C090E090939F0285E089
:10243000891B80938A020E9488118AE0E5E9F2E014
:10244000DF01982F1D929A95E9F7EBE8F2E0DF01A2
:102450001D928A95E9F785E00E9484120C9411027E
:10246000EF92FF920F931F93CF93DF93CDB7DEB719
:102470002A970FB6F894DEBF0FBECDBF8E010F5F57
:102480001F4F8AE0F80111928A95E9F7F12C6F2D20
:10249000C8010E94A811F394F5E0FF12F8CF4AE0BA
:1024A00050E0B8018BE892E00E9477247C0121E0A3
:1024B000892B09F420E0E114F10441F08AE0F801ED
:1024C000ABE8B2E001900D928A95E1F760919F022E
:1024D00070E06B567D4F45E08BE892E00E948512DC
:1024E000EF2819F40E940B1102C081E090E02A96B7
:1024F0000FB6F894DEBF0FBECDBFDF91CF911F9115
:102500000F91FF90EF9008950895FF920F931F93FE
:10251000CF93DF938C01F62ED72FC42F222349F0BF
:1025200081E080933D020E94F11C90933C028093D5
:102530003B0280913D028823C1F080913B02909143
:102540003C020E94091D059780F0EF2DFD2FD80158
:102550004C2F50E0CD01801B910B841795071CF484
:102560008D918193F7CF10923D02DF91CF911F9112
:102570000F91FF90089584988C988FB18295817007
:1025800008958091400281110DC00E943C24811168
:1025900002C082E001C081E080934002823011F4E9
:1025A0000E94372481E090914002913009F080E050
:1025B00008950E94BB12809304010E94C1128111F0
:1025C0000C94291308950E94C112811102C00C9429
:1025D0002B13089581E0909141029A3008F080E039
:1025E00008950F931F93CF93DF93EC018B0180919C
:1025F00041028A3038F4B801CE010E94791381116A
:102600001DC00AC080913E0290913F020E94091DA8
:10261000843F914080F715C0809141028F3F19F0AF
:102620008F5F80934102809141028A3060F00E9466
:10263000F11C90933F0280933E0203C0109241022E
:1026400002C080E001C081E0DF91CF911F910F9126
:1026500008950C94401A0C94431ADF92EF92FF9263
:102660000F931F93CF93DF937901C82F880FDD0B52
:1026700041155105A9F0FE0193E0EE0FFF1F9A9559
:10268000E1F7EB5FFE4F818192818E5B9D4F208150
:1026900030E04217530708F49A01A9010E948424EC
:1026A000CE010E942C1BD82E8823D1F001151105D4
:1026B000B9F083E0CC0FDD1F8A95E1F7FE01EB5FF7
:1026C000FE4F438150E00417150708F4A801CB5FC3
:1026D000DE4F6C817D816E5B7D4FC7010E9484243B
:1026E0008D2DDF91CF911F910F91FF90EF90DF9093
:1026F00008950C9495140C94B1140F931F93CF93D9
:10270000DF9300D000D0CDB7DEB760915902709151
:102710005A0280915B0290915C020E94181D6436FF
:1027200071058105910528F10E949810DC01CB010B
:102730000296A11DB11D89839A83AB83BC8300E0FF
:1027400010E020E030E044E050E0BE016F5F7F4FDA
:1027500082E00E942D13182F882361F00E94FD1C37
:102760006093590270935A0280935B0290935C02CB
:1027700001C011E0812F0F900F900F900F90DF910B
:10278000CF911F910F910895AF92BF92CF92DF9298
:10279000EF92FF920F931F93CF93DF937C015B0126
:1027A0006A010E94EA12811103C001E010E002C038
:1027B0000AE010E0C1E0D0E0F894B501C701F601ED
:1027C00009957894811115C021960C171D0794F076
:1027D000CC9F9001CD9F300D300D112480E090E012
:1027E00045E34A95F1F70000019682179307C1F778
:1027F000E3CF81E0DF91CF911F910F91FF90EF9098
:10280000DF90CF90BF90AF900895AF92BF92CF92DC
:10281000DF92EF92FF920F931F93CF93DF9300D03D
:1028200000D000D0CDB7DEB77B01C090A001D09022
:10283000A10101E010E09E012A5F3F4F40E050E01F
:1028400060E070E080E00E942D13182F882309F4C7
:102850003EC056018FEFA81AB80A609155027091D8
:10286000560280915702909158020E94181D6436BA
:1028700071058105910518F105E010E09E012F5FBB
:102880003F4F40E050E060E070E081E00E942D1397
:10289000182F65E070E0C5010E948E1791E02E812F
:1028A000281390E0192339F10E94FD1C6093550212
:1028B00070935602809357029093580211C065E0BE
:1028C00070E0C5010E948E179E818913D5CF85E0E7
:1028D000F6013196DE01119601900D928A95E1F78D
:1028E000112349F085E0FE013196A0E5B2E00190A8
:1028F0000D928A95E1F785E0E0E5F2E0D7010190DD
:102900000D928A95E1F7812F26960FB6F894DEBFD7
:102910000FBECDBFDF91CF911F910F91FF90EF9030
:10292000DF90CF90BF90AF9008950F931F93CF93F8
:10293000DF93EC018B0145E054E10E94C41388232E
:1029400051F04DE753E1B801CE01DF91CF911F91D6
:102950000F910C94C41380E0DF91CF911F910F91E0
:1029600008950F931F93CF93DF93F894C091A00124
:10297000D091A101CE01019625E0FB01DC0101907F
:102980000D922A95E1F765E070E00E948E1788832A
:102990007894F8946E817F818885998500914C02A6
:1029A00010914D0220914E0230914F026017710735
:1029B0008207930751F060934C0270934D0280930D
:1029C0004E0290934F020E947B107894DF91CF913A
:1029D0001F910F9108950E94FD1E0E94D30D0C942B
:1029E000091F0E940D1F0E94690E0C94271F0E9450
:1029F0008F1C0E94E41E0E94C10D0E94EB140E94D5
:102A0000F1140E94CB0DFBCF8091630280FF06C0C2
:102A10006091220170E0660F771F26C081FF04C01D
:102A20006091220184E005C082FF07C0609122010D
:102A300088E0689FB001112417C090916202992329
:102A4000D1F060912101961788F72091220188E04A
:102A5000289F90011124929FA001939F500D112453
:102A600070E0CA010E9449246038710540F4611584
:102A7000710519F406C068E070E0862F08958FE7AD
:102A8000089581E008958091630280FF08C06091FD
:102A90001E0170E0759567957595679521C081FF5A
:102AA00006C060911E0170E07595679519C082FFA0
:102AB00004C060911E0170E010C0909161029923E2
:102AC00099F060911D019617A0F780911E01899FD2
:102AD000C001112470E00E9449246038710540F45F
:102AE0006115710519F406C061E070E0862F089544
:102AF0008FE7089581E008958D3E21F40E9404152A
:102B0000819504C08E3E29F40E94041580936702CB
:102B100008958F3E21F40E940415819504C0803FE2
:102B200029F40E940415809366020895893F19F4E0
:102B30000E94431505C08A3F31F40E9443158195D8
:102B40008093680208958B3F21F40E94431581957C
:102B500004C08C3F29F40E944315809369020895B4
:102B60009FE0980F983078F421E030E0A90102C08E
:102B7000440F551F9A95E2F7CA0190916502892B7F
:102B80008093650208958D3F21F4809163028160F6
:102B90000BC08E3F21F480916302826005C08F3F9D
:102BA00029F48091630284608093630208958D3ECE
:102BB00039F49091670297FF35C01092670259C0AF
:102BC0008E3E29F4909167021916BCF32BC09091A8
:102BD00066028F3E29F497FF25C01092660249C015
:102BE000803F19F41916CCF31DC090916802893FFB
:102BF00029F41916BCF4109268023BC08A3F19F4FC
:102C000097FF10C0F8CF8B3F39F49091690297FF7E
:102C100009C0109269022DC08C3F21F49091690285
:102C20001916BCF39FE0980F983080F421E030E053
:102C3000A90102C0440F551F9A95E2F7CA01809579
:102C40009091650289238093650213C08D3F21F422
:102C5000809163028E7F0BC08E3F21F480916302CE
:102C60008D7F05C08F3F29F4809163028B7F809315
:102C7000630280916602811106C080916702811112
:102C800002C01092620280916802811106C0809198
:102C90006902811102C01092610208950E94F11C24
:102CA00020916602211104C020916702222321F0A5
:102CB0009093600280935F0220916802211104C00A
:102CC00020916902222321F090935E0280935D029D
:102CD00084E692E00C94CF1BEF92FF920F931F9328
:102CE000CF93DF9300D000D000D0CDB7DEB786E021
:102CF000E4E6F2E0DE01119601900D928A95E1F78B
:102D0000E0906602F09067020091680210916902FB
:102D10001092660210926702109268021092690285
:102D2000E11003C0FF2009F45DC080915F02909123
:102D300060020E94091DAC0190916202992339F052
:102D40002091230130E02417350758F04BC0209123
:102D500024018AE0289F900111242417350718F0D8
:102D600041C09F3F19F09F5F90936202EE2061F097
:102D70000E9404151E1414F09FEF01C091E0989F6B
:102D8000902D112490936602FF2061F00E9404159B
:102D90001F1414F09FEF01C091E0989F902D112413
:102DA00090936702309166023323E1F0209167022D
:102DB0002223C1F045EB3403C0011124992319F0FB
:102DC0009093660203C081E08093660235EB230393
:102DD000C0011124992319F09093670203C081E088
:102DE00080936702011103C0112309F45DC0809133
:102DF0005D0290915E020E94091DAC0190916102FA
:102E0000992339F020911F0130E02417350758F03D
:102E10004BC0209120018AE0289F900111242417A3
:102E2000350718F041C09F3F19F09F5F90936102F2
:102E3000002361F00E944315101614F09FEF01C0AB
:102E400091E0989F902D112490936802112361F0D6
:102E50000E944315111614F09FEF01C091E0989F56
:102E6000902D112490936902309168023323E1F090
:102E7000209169022223C1F045EB3403C0011124E3
:102E8000992319F09093680203C081E0809368024F
:102E900035EB2303C0011124992319F090936902A3
:102EA00003C081E0809369028091660281110BC0AA
:102EB00080916702811107C080916802811103C06F
:102EC0008091690281110E944E16EB82FC820D8373
:102ED0001E8386E0FE013196A4E6B2E001900D92D9
:102EE0008A95E1F726960FB6F894DEBF0FBECDBFE8
:102EF000DF91CF911F910F91FF90EF900895E4E63D
:102F0000F2E086E0DF011D928A95E9F710926202F5
:102F1000109261021092630208950895FC01680FF7
:102F2000791F8FEF91E3E617F70771F02191822760
:102F300028E030E087FF03C0880F892701C0880F91
:102F400021503109B9F7EFCF0895CF93DF93EC010A
:102F5000FB018281882309F43CC1C430FDE5DF0711
:102F600060F4CB3F9CE5D90788F49E0122503C4594
:102F70002431310508F02EC109C0C236EDE5DE0767
:102F800029F0C63AFDE5DF0709F024C10E94FC0CD8
:102F90009093890280938802C1318CE5D80709F4A7
:102FA000C6C008F042C0C930ECE5DE0709F49BC09A
:102FB00000F5C5308CE5D80709F485C078F4C33036
:102FC000ECE5DE0709F478C008F07AC0C230DC45D1
:102FD00009F0F5C0809188028160EFC0C7309CE5A0
:102FE000D90709F478C008F07AC08091880280611E
:102FF000E4C0CD30FCE5DF0709F487C058F4CB30DE
:103000009CE5D90709F479C008F07BC0809188025B
:1030100088606FC0CF30FCE5DF0709F480C008F09E
:1030200082C080918802877FC8C0CE3F9CE5D907C7
:1030300009F471C000F5C531FCE5DF0709F485C06E
:1030400068F4C3319CE5D90709F475C008F095C050
:103050000E94C706809188028F77AFC0CC3FFCE505
:10306000DF07A9F108F054C0CB3FDC4509F0A7C049
:103070008091890240C0C230EDE5DE0709F489C0C5
:1030800058F4C1158DE5D80709F45AC008F069C095
:103090008091890282602FC0C236EDE5DE0709F417
:1030A0007CC0C63AFDE5DF0709F481C0C330DD45C9
:1030B00009F085C080E06EC08091880282607DC08A
:1030C0008091880216C080918802886076C08091C5
:1030D000890282604FC08091880280626EC08091B8
:1030E000880280646AC00E94C70680918802806856
:1030F00064C0846062C081603DC0809188028E7F20
:103100005CC0809188028D7F58C08091880216C073
:103110008091890218C0809189028D7F2BC0809197
:1031200088028F7E4AC0809188028F7D46C0809140
:1031300088028F7B42C080918802877F8B7F3DC051
:10314000809189028D7F8E7F15C08091880282FBDD
:10315000222720F991E0922790FB82F990FB83F9D6
:103160002CC080918902982F909591708E7F892B29
:1031700090FB81F98093890222C00E94C70680914A
:10318000880287FB222720F991E0922790FB87F99C
:1031900014C081E00E94930D12C08091880284FBCC
:1031A000222720F991E0922790FB84F906C08091B4
:1031B0008802982F909590FB80F9809388028091E7
:1031C0008802909189020E940D0D0E94C70680E03E
:1031D00001C081E0DF91CF910895CF93DF938631D5
:1031E0009C4541F5EB010E94000C982F8A812091AB
:1031F000020130910301882379F09A7A81E009F481
:1032000080E080936A02911102C069E201C065E327
:10321000C9010E944B1C0AC080916A02811102C040
:1032200069E201C065E3C9010E944D1C0E94420C85
:1032300080E001C081E0DF91CF9108950F931F934B
:10324000CF93DF93C42FD22FFC0182818823C9F052
:1032500040936D020E94F11C90936C0280936B026C
:1032600080E28C0F883008F057C0C77081E001C041
:10327000880FCA95EAF7DF91CF911F910F910C94B7
:10328000240480916D02481330C080916B029091AC
:103290006C020E94091D843B910538F510E21D0F58
:1032A000CD17B9F080E28C0F883040F4C77081E010
:1032B00001C0880FCA95EAF70E942B04183028F540
:1032C00081E09D2F977001C0880F9A95EAF70E94C0
:1032D0002404802F0E941B041830F0F4D77081E082
:1032E00001C0880FDA95EAF70AC080E28C0F8830B7
:1032F00098F4C77081E001C0880FCA95EAF7DF91A2
:10330000CF911F910F910C942B04802FDF91CF91BF
:103310001F910F910C941B04DF91CF911F910F917E
:1033200008950F939C01CB01243F4CE5340731F104
:1033300088F4293DFCE53F07D9F02A3D4CE53407E8
:1033400079F1283D3C45A9F506E221EE41EE68ED14
:103350007CE52BC0263FFCE53F07E1F0A8F0273FC6
:103360003C4539F507E225EE46EE67EF7CE51DC0EA
:1033700007E225EE45EE69ED7CE517C006E221EE99
:1033800040EE64EF7CE511C007E225EE44EE65EF08
:103390007CE50BC006E221EE42EE66EF7CE505C05F
:1033A00008E221E045EE6AED7CE50E941E1980E00E
:1033B00008C0FC018281882319F010926D0201C0BF
:1033C00081E00F9108958EE14A9B02C08150E1F7A0
:1033D0004A9BFECF08955A9880E28A95F1F75A9A4F
:1033E0000895FC012AE02A95F1F728E090E080E0BA
:1033F00031E040E14A95F1F7880F4A9B02C08160B5
:10340000932700C0000040E14A95F1F7215089F769
:1034100020E12A95F1F729B100C0000030E13A958A
:10342000F1F722FB222720F992272081920F908327
:103430000895EF92FF920F931F93CF93DF931F9204
:10344000CDB7DEB719828C017C01E60EF11C0E159A
:103450001F0551F00E94E319CE0101960E94F11957
:10346000F80181938F01F3CF81E09981911180E080
:103470000F90DF91CF911F910F91FF90EF900895E2
:10348000529A5A9A089552985A9AEA9AE9E6F0E0BE
:1034900080818F7C80830895615091E001C0990FF5
:1034A0006A95EAF720E031E0992361F0492F48233B
:1034B00019F05A9A232701C05A9840E24A95F1F729
:1034C0009695F2CF222311F05A9A01C05A9880E2C1
:1034D0008A95F1F75A980895FF920F931F93CF930F
:1034E000DF93EC018C01060F111DC017D10741F0CD
:1034F000F9900E94EB1968E08F2D0E944C1AF5CFCD
:10350000DF91CF911F910F91FF9008951F920F921D
:103510000FB60F9211240F931F932F933F934F9346
:103520005F936F937F938F939F93AF93BF93EF932B
:10353000FF93CF93DF931F92CDB7DEB719820E941E
:10354000E319CE0101960E94F119082F0695069500
:103550000695902F96959570202F2570920F292F04
:10356000237096959695920F877089135FC0898115
:1035700081115CC0043008F059C080E18A95F1F7F0
:103580005A9A529A82E08A95F1F700C05A9888E0D8
:10359000089F80011124D801AB5FBE4F1696ED91B4
:1035A000FC9117973097A9F06091A0017091A1014B
:1035B00014962D913C911597260F371F11968D91DA
:1035C0009C911297680F791F13964C9113978C91C9
:1035D0000995F801EB5FFE4F6381662351F08091FE
:1035E000A0019091A10124813581820F931F0E9437
:1035F0006C1A0E94EB1980E18A95F1F75A9852985B
:103600005A9A80E18A95F1F7F801EB5FFE4F6081ED
:10361000662351F08091A0019091A1012181328116
:10362000820F931F0E94191A0E94E3190F90DF91D5
:10363000CF91FF91EF91BF91AF919F918F917F912A
:103640006F915F914F913F912F911F910F910F902B
:103650000FBE0F901F9018950F931F93CF93DF937A
:10366000843091050CF06DC0EC01F894529A5A9890
:1036700085E08A95F1F700009C2F969595702C2F88
:103680002570920F892F83709695969523E0CC0F25
:10369000DD1F2A95E1F7980F8E01092B0E94EB1987
:1036A00084E08A95F1F700C068E0802F0E944C1AF0
:1036B00080E18A95F1F752985A9A4A9902C000C05F
:1036C000FCCF87E090E04A9B08C0019721F4529A12
:1036D0005A9A789436C000C0F6CFFE01EB5FFE4FD9
:1036E0006381662381F08091A0019091A1012481E2
:1036F0003581820F931F0E94191A811104C0529ABA
:103700005A9A78941FC00E94E31980E28A95F1F7D3
:103710005A98529A80E18A95F1F7CB5FDE4F688123
:10372000662351F08091A0019091A10129813A81F5
:10373000820F931F0E946C1A0E94EB19789481E00B
:1037400001C080E0DF91CF911F910F910895909378
:10375000A3018093A2010895909374028093730251
:1037600008950E94C112811103C080916E020895D4
:10377000E0917302F0917402309721F00190F08192
:10378000E02D099480E00895E0917302F0917402B5
:10379000309721F00280F381E02D09940895E091A3
:1037A0007302F0917402309739F022E0DC012C931F
:1037B0000480F581E02D09940895209171023091E3
:1037C00072022817390771F0909372028093710288
:1037D000E0917302F0917402309721F00680F78136
:1037E000E02D0994089520916F02309170022817FE
:1037F000390771F09093700280936F02E091730229
:10380000F0917402309721F00084F185E02D099445
:103810000895FC01329697E080E0915029F02191C3
:103820002223D9F38F5FF9CF0895662349F0FC0175
:10383000329608962191621729F0E817F907D1F717
:1038400080E0089581E008959C01FC0132969FEF8D
:1038500080E04191461789F09F3F19F4411101C062
:10386000982F8F5F8630A9F79F3F39F0F901E90F54
:10387000F11D97FDFA956283089508959C012A5FD2
:103880003F4FFC014281461301C01282019682170C
:103890009307B9F708950C94241C0C943E1C0296CF
:1038A00026E0FC0111922A95E9F7089508950C94F9
:1038B000561C83E0809375020C94571C811102C042
:1038C00081E001C082E0809375020C94571C0C9437
:1038D0005E1C81E0809375020C94571C0C94691C4B
:1038E00008950C94701C0C94711C0C94701C0C9416
:1038F000701C0C94701CCF930E94771C0E94301295
:103900000E94751CC0E08C2F0E94F110811104C030
:10391000CF5FCA30C1F701C081E0CF91089508950B
:103920001F920F920FB60F9211248F939F93AF9314
:10393000BF9380917602811113C08091A002909173
:10394000A102A091A202B091A3024196A11DB11DB6
:103950008093A0029093A102A093A202B093A3022D
:10396000BF91AF919F918F910F900FBE0F901F90BD
:1039700018958091A802843031F10E94770210924C
:10398000760220E488E190E00FB6F894A895809341
:1039900060000FBE2093600083B7817F846083BF87
:1039A00083B7816083BF7894889583B78E7F83BF08
:1039B0000FB6F894A89580916000886180936000AC
:1039C000109260000FBE08950E94C7060C947B02FF
:1039D00082E084BD93E095BD9AEF97BD80936E0021
:1039E00008952FB7F8948091A0029091A102A09120
:1039F000A202B091A3022FBF08952FB7F89460914F
:103A0000A0027091A1028091A2029091A3022FBF07
:103A100008959C014FB7F8948091A0029091A10263
:103A2000A091A202B091A3024FBF821B930B0895F5
:103A3000CF92DF92EF92FF922FB7F894C090A0023E
:103A4000D090A102E090A202F090A3022FBFA701A4
:103A50009601261B370B480B590BCA01B901FF9081
:103A6000EF90DF90CF90089578941F920F920FB649
:103A70000F9211248F939F93AF93BF938091A002D5
:103A80009091A102A091A202B091A3020196A11D62
:103A9000B11D8093A0029093A102A093A202B093C3
:103AA000A302BF91AF919F918F910F900FBE0F9086
:103AB0001F90189587E797E7909301088093000877
:103AC0009AE088E10FB6F894A895809360000FBE45
:103AD00090936000FFCF809182020895089522E0C4
:103AE0002093E9002FEF3091E800215035FD06C00A
:103AF00035ED3A95F1F700002111F5CF2091E8005E
:103B000025FF0BC040E050E066E070E00E94991F86
:103B10008091E8008E778093E8000895CF93DF933B
:103B200021E02093E9002FEF3091E800215035FD8E
:103B300006C035ED3A95F1F700002111F5CF20913F
:103B4000E80025FF14C0EC0140E050E068E070E0C0
:103B50000E94991F8091E8008E778093E80088E0AA
:103B6000FE01AAE7B2E001900D928A95E1F7DF919C
:103B7000CF910895809377027093790260937802D1
:103B80008091A802843001F582E08093E9008FEFF4
:103B90009091E800815095FD06C095ED9A95F1F75A
:103BA00000008111F5CF8091E80085FF0DC040E055
:103BB00050E063E070E087E792E00E94991F8091F7
:103BC000E8008E778093E8000895BC0184E00C94AF
:103BD000BA1DBC0183E00C94BA1D8091A70281112B
:103BE00009C00E942A210E9487218091E2008460FE
:103BF0008093E20008951092A70208950C946E1C21
:103C00006091A40281E0611101C080E00C94591C14
:103C10009091A80281E0943009F080E06091A402C4
:103C20000C945E1C42E061EC81E00E94A32042E221
:103C300061EC82E00E94A3209091A80281E0943080
:103C400009F080E06091A4020C94671C8091AA02A4
:103C5000833009F461C030F4813071F0823009F4AE
:103C60009AC008958A3009F486C08B3009F46CC07C
:103C7000893009F0A8C020C08091A902813A09F0DA
:103C8000A2C08091E800877F8093E8008091AD0218
:103C90009091AE02892B21F468E08AE792E003C09C
:103CA00060E080E090E070E00E94E41F8091E80016
:103CB0008B778093E80008958091A902813209F002
:103CC00082C08091AD029091AE02029708F07BC055
:103CD0008091E800877F8093E8008091E80082FD72
:103CE00005C08091A8028111F8CF6DC02091F3002A
:103CF0008091F20090E0922B029731F48091F100D4
:103D0000813011F0863021F48091F100809382029D
:103D10008091E8008B7753C08091A902813A09F025
:103D200052C08091AD029091AE02892B09F04BC038
:103D30008091E800877F8093E8008091E80080FF11
:103D4000FCCF8091310136C08091A9028132D9F532
:103D50008091AD029091AE02892BA9F58091E80087
:103D6000877F8093E8000E94D8208091AB028093E7
:103D700031010C94C7068091A902813221F580910E
:103D8000E800877F8093E8000E94D8208091AC02F1
:103D90008093830208958091A902813AA1F48091D1
:103DA000E800877F8093E8008091E80080FFFCCFE7
:103DB000809183028093F1008091E8008E77809358
:103DC000E8000C94D820089584B7877F84BF0FB68D
:103DD000F894A895809160008861809360001092AB
:103DE00060000FBE90E080E80FB6F8948093610009
:103DF000909361000FBE0C94691C0E942A210E94BE
:103E00008721E2EEF0E080818460808378940C94D6
:103E10001C2485E291E00C94AC1B8091A8028530B3
:103E2000A9F48091A802853079F40E94B91C809190
:103E3000A6028823B1F30E947B1C882391F30E9481
:103E4000831F0E94C706EDCF0C94E41C08950895CB
:103E50000C942A1F292F332723303105C9F060F431
:103E60002130310581F02230310509F044C08BE367
:103E700090E028E332E043C021323105E1F0223204
:103E8000310549F138C082E190E023E732E037C0E4
:103E900099278130910549F028F0029761F5E0EF0C
:103EA000F1E005C0E4E3F2E002C0E6E0F2E0849174
:103EB00090E09F0124C06115710541F061307105EA
:103EC000D1F489E090E023E632E019C089E090E087
:103ED0002AE432E014C06115710541F061307105CA
:103EE00051F48BE790E025E832E009C080E490E0EF
:103EF00020E033E004C080E090E020E030E0FA0110
:103F000031832083089580E189BD82E189BD09B4B0
:103F100000FEFDCF8091D8008F7D8093D8008091E6
:103F2000E00082608093E0008091E00081FDFCCFA2
:103F30000895CF92DF92EF92FF920F931F93CF934A
:103F4000DF93EC018B017A010E94F720811133C0CD
:103F5000E114F10439F0F70180819181081B190BFC
:103F6000C80FD91FC12CD12C0115110519F1809151
:103F7000E80085FD16C08091E8008E778093E80008
:103F8000E114F10449F0F70180819181C80ED91E36
:103F9000D182C08285E00FC00E94F720882321F3E0
:103FA0000AC089918093F10001501109FFEFCF1AE7
:103FB000DF0ADACF80E0DF91CF911F910F91FF9060
:103FC000EF90DF90CF9008952091AF023091B00232
:103FD0002617370748F06115710539F42091E8007C
:103FE0002E772093E80001C0B901FC0120E06115A3
:103FF000710579F18091A8028823F1F18530F1F102
:104000008091E80083FD3CC08091E80082FD2EC0D5
:104010008091E80080FFEBCF2091F3008091F200C7
:1040200090E0922B6115710551F08830910538F4BC
:1040300021912093F100615071090196F3CF21E0A5
:10404000089709F020E08091E8008E778093E800DF
:10405000CECF2111CFCF0AC08091A802882361F072
:10406000853061F08091E80083FD0AC08091E8000E
:1040700082FFF2CF80E0089582E0089583E0089502
:1040800081E008952091AF023091B00226173707E2
:1040900048F06115710539F42091E8002E772093DE
:1040A000E80001C0B901FC0120E06115710591F142
:1040B0008091A802882309F440C0853009F43FC0EC
:1040C0008091E80083FD3DC08091E80082FD2FC013
:1040D0008091E80080FFE9CF2091F3008091F20009
:1040E00090E0922B6115710559F08830910540F4EC
:1040F00024912093F1003196615071090196F2CF1D
:1041000021E0089709F020E08091E8008E77809305
:10411000E800CBCF2111CCCF0AC08091A802882320
:1041200061F0853061F08091E80083FD0AC08091E4
:10413000E80082FFF2CF80E0089582E0089583E0F6
:10414000089581E00895982F973068F59093E900DD
:10415000981739F07091EC002091ED005091F0002B
:1041600003C0242F762F50E021FD02C09F5FECCFCB
:104170003091EB003E7F3093EB003091ED003D7FBE
:104180003093ED003091EB0031603093EB00709391
:10419000EC002093ED005093F0002091EE0027FDFD
:1041A000E5CF80E008958F708093E90081E0089565
:1041B0008091A90287FF11C08091E80082FD05C0AF
:1041C0008091A8028111F8CF11C08091E8008B770F
:1041D0000BC08091A802882349F08091E80080FFFD
:1041E000F8CF8091E8008E778093E80008952091C1
:1041F000E4003091E50095E64091EC00842F817059
:1042000040FF23C08091E80080FD1DC08091A8027E
:10421000882399F0853099F08091EB0085FD11C0DD
:104220004091E4005091E5002417350729F391509F
:1042300011F09A01E1CF84E0089582E0089583E0CF
:10424000089581E0089580E008954091E80042FFDC
:10425000DDCF08950E9498210E94A021E0EEF0E0B9
:10426000808181608083E8EDF0E080818F778083BA
:1042700019BCA7EDB0E08C918E7F8C9380818F7EEE
:1042800080831092A70208950F931F93CF93DF931B
:104290000E9498210E94A021C8EDD0E088818F77EC
:1042A000888388818068888388818F7D888319BC12
:1042B0001092A8021092A4021092A6021092A502D7
:1042C00000EE10E0F80180818B7F8083888181601F
:1042D000888342E060E080E00E94A320E1EEF0E00D
:1042E00080818E7F8083E2EEF0E080818160808338
:1042F000808188608083F80180818E7F80838881BF
:1043000080618883DF91CF911F910F910895E8ED2F
:10431000F0E080818F7E8083E7EDF0E08081816036
:10432000808384E082BF81E08093A7020C944421C3
:10433000E8EDF0E080818E7F80831092E2000895A6
:104340001092DA001092E10008951F920F920FB6BA
:104350000F9211242F933F934F935F936F937F930B
:104360008F939F93AF93BF93EF93FF938091E1005F
:1043700082FF0BC08091E20082FF07C08091E100C4
:104380008B7F8093E1000E941B248091DA0080FFE4
:104390001FC08091D80080FF1BC08091DA008E7F03
:1043A0008093DA008091D90080FF0DC080E189BD43
:1043B00082E189BD09B400FEFDCF81E08093A802AF
:1043C0000E94ED1D05C019BC1092A8020E94FB1DA1
:1043D0008091E10080FF19C08091E20080FF15C04C
:1043E0008091E2008E7F8093E2008091E200806104
:1043F0008093E2008091D80080628093D80019BC3D
:1044000085E08093A8020E94001E8091E10084FF55
:1044100030C08091E20084FF2CC080E189BD82E140
:1044200089BD09B400FEFDCF8091D8008F7D8093B7
:10443000D8008091E1008F7E8093E1008091E200BE
:104440008F7E8093E2008091E20081608093E200A1
:104450008091A402882311F084E007C08091E300DA
:1044600087FD02C081E001C083E08093A8020E9422
:10447000081E8091E10083FF29C08091E20083FF44
:1044800025C08091E100877F8093E10082E08093E6
:10449000A8021092A4028091E1008E7F8093E10037
:1044A0008091E2008E7F8093E2008091E200806143
:1044B0008093E20042E060E080E00E94A3208091CF
:1044C000F00088608093F0000E94FE1DFF91EF9144
:1044D000BF91AF919F918F917F916F915F914F911C
:1044E0003F912F910F900FBE0F901F9018951F9224
:1044F0000F920FB60F9211242F933F934F935F9318
:104500006F937F938F939F93AF93BF93CF93DF93DB
:10451000EF93FF93C091E900CF708091EC00D82F0A
:10452000D17080FDD0E81092E9008091F000877F83
:104530008093F00078940E94BB221092E900809151
:10454000F00088608093F000CD2BCF70C093E9001D
:10455000FF91EF91DF91CF91BF91AF919F918F919B
:104560007F916F915F914F913F912F910F900FBE6F
:104570000F901F9018951F93CF93DF93CDB7DEB7A1
:10458000AA970FB6F894DEBF0FBECDBFE9EAF2E0FE
:104590008091F100819322E0E13BF207C9F70E948C
:1045A000261E8091E80083FF2EC18091A902909180
:1045B000AA02492F50E04A30510508F024C1FA01FF
:1045C000EE59FF4F0C945D24803821F0823809F0B9
:1045D0001AC108C08091A5029091A602992389F082
:1045E00082600FC08091AD028F70873008F00BC1E0
:1045F0008093E9008091EB0085FB882780F9109279
:10460000E9009091E800977F9093E8008093F10093
:104610001092F100D1C0282F2D7F09F0F4C088231B
:1046200019F0823061F0EFC08091AB02813009F067
:10463000EAC0933009F080E08093A6022EC08091FA
:10464000AB0281112AC08091AD028F702FEF280F2D
:10465000263008F0D8C08093E9002091EB0020FFBD
:104660001CC0933021F48091EB00806214C09091C3
:10467000EB0090619093EB0021E030E0A90102C0D3
:10468000440F551F8A95E2F74093EA001092EA0022
:104690008091EB0088608093EB001092E90080919C
:1046A000E800877F8093E8000E94D820ACC0811189
:1046B000AAC01091AB021F778091E3008078812B14
:1046C0008093E3008091E800877F8093E8000E9458
:1046D000D8208091E80080FFFCCF8091E3008068C3
:1046E0008093E300111102C082E001C083E0809357
:1046F000A80289C08058823008F085C08091AB0242
:104700009091AC028C3D53E0950779F583E08A8364
:104710008AE289834FB7F894DE01139620E03EE0E9
:1047200051E2E32FF0E050935700E49120FF03C0E3
:10473000E295EF703F5FEF708E2F90E0EA3010F05F
:10474000C79601C0C0968D939D932F5F243149F782
:104750004FBF8091E800877F8093E8006AE270E0B5
:10476000CE0101960E94E41F16C06091AD027091C7
:10477000AE02AE014F5F5F4F0E94281FBC01892B24
:1047800009F441C09091E800977F9093E8008981F7
:104790009A810E9442208091E8008B778093E80004
:1047A00032C0803881F58091E800877F8093E800EF
:1047B0008091A4028093F1008091E8008E7772CFFF
:1047C000811121C08091AB029091AC029927029790
:1047D000D4F48091E800877F8093E8008091AB0259
:1047E0008093A4020E94D8208091A402811106C067
:1047F0008091E30087FD02C081E001C084E08093E6
:10480000A8020E94121E8091E80083FF0AC08091D6
:10481000E800877F8093E8008091EB0080628093BE
:10482000EB00AA960FB6F894DEBF0FBECDBFDF91A6
:10483000CF911F9108950895CF938091A802882366
:10484000A1F0C091E900CF709091EC00892F8170A8
:1048500090FD80E8C82B1092E9008091E80083FD6C
:104860000E94BB22CF70C093E900CF9108950E94AF
:104870002A211092A8020895E8EDF0E0808180617D
:1048800080838AE18A95F1F700C08091D900817018
:10489000089597FB072E16F4009407D077FD09D0F2
:1048A0000E94632407FC05D03EF4909581959F4FAC
:1048B0000895709561957F4F0895EE0FFF1F059045
:1048C000F491E02D0994AA1BBB1B51E107C0AA1F5C
:1048D000BB1FA617B70710F0A61BB70B881F991FA1
:1048E0005A95A9F780959095BC01CD010895FB01DB
:1048F000DC0104C08D910190801921F44150504099
:10490000C8F7881B990B0895FB01DC0102C00190D8
:104910000D9241505040D8F70895F999FECF92BDBD
:1049200081BDF89A992780B50895A8E1B0E042E0EA
:1049300050E00C94C124262FF999FECF92BD81BD81
:10494000F89A019700B4021639F01FBA20BD0FB6CD
:10495000F894FA9AF99A0FBE08950396272F0E94A9
:104960009C240E949B24252F0E949C24242F0C947D
:104970009C240196272F0E949C240C949B24DC01EC
:10498000CB01FC01F999FECF06C0F2BDE1BDF89A5A
:10499000319600B40D9241505040B8F70895F89404
:0249A000FFCF47
:1049A200B4001D0201000000010000000000000030
:1049B2000501000000040600000000000028085065
:1049C200011E0A14016B1D8E1D6F1DE91DE51D6E72
:1049D2001D01E200E900EA00B500B600B700CD0013
:1049E2008301CC008A019201940121022302240254
:1049F2002502260227022A02B300B4006F007000CB
:104A0200818283E200E900EA00B500B600B700CD7A
:104A1200008301CC008A0192019401210223022425
:104A2200022502260227022A02B300B4006F007098
:104A320000818283F5F6F7313332366697C6343514
:024A420042022E
:00000001FF
